:020000040000FA
:020000003B289B
:080008008C00030E8D008B1A21
:100010000B1D0D281E200B1119280B1A8B1C1328E1
:1000200032208B1019288B190B1C19283A200B1021
:1000300019280D0E83008C0E0C0E090064000000C0
:1000400000009D10D03081009D168613910AA00BF0
:100050002B280510A103851C8617061C31281D1F9F
:100060009D140800010890001108930091011D17CC
:100070001D14080008008501860183168901C2301D
:1000800081000C3084008001840A041F4328041E70
:100090004328E2308500733086008312FF30A100D0
:1000A000910ACD308100B2308B00E62064001D182B
:1000B000612021080319FE209D1A1A21061C1D1318
:1000C0005628132133211D101930A100A31C952897
:1000D00005101208CD3C031879281D1E7628061538
:1000E00086110514CD30120295008C281D169D1125
:1000F0008C2803101208AA3C031C92289D1D8A28F4
:100100008615061105140310AA301202031C003CC8
:1001100095008C281D129D151508A0000310150CC4
:10012000A007D82886110611D828231DB72817083C
:100130000F3997001208643C0318B5281208913C47
:10014000031CA4281717B5281208AA3C031CAA28C8
:100150009717B5281208C53C031CB0281716B528F8
:100160001208DC3C031CB5289716DA20D828A31DFA
:10017000D8281708F03997001208643C0318B528EE
:100180001208913C031CC6281714B5281208AA3C73
:10019000031CCC289714B5281208C53C031CD22890
:1001A0001715B5281208DC3C031CB5289715B5288F
:1001B0001D1108001A081902031DF6281908180253
:1001C000031DF62818081702031DF62817089500C6
:1001D00008309400151CEE280515EF2805110516AA
:1001E0000512950C940BEA288515851119089A00BB
:1001F0001808990017089800051108001D190F2903
:1002000017179713E6201430A10064002108031D7E
:1002100005299701E6200510861106111D15A2017A
:10022000A3016300080001089400010814020319E7
:10023000152908009D1206183229861E2229061C3F
:10024000A3142429061CA310061E2929061C231505
:100250002B29061C2311861C3029061CA3153229C4
:10026000061CA31108009303CD301002031C32308A
:1002700090000F08323C1007323E03184229930BBE
:100280003C294329FF3092009D1F4C29043012075E
:100290000318FF3092009D139D1C512904309202D7
:0802A0009D1710088F000800F3
:02400E00F63F7B
:00000001FF
